:100000000C9434000C9451000C9451000C94510049
:100010000C9451000C9451000C9451000C9451001C
:100020000C9451000C9451000C9451000C9451000C
:100030000C9451000C9451000C9451000C945100FC
:100040000C9451000C9451000C9451000C945100EC
:100050000C9451000C94D8000C9451000C94510055
:100060000C9451000C94510011241FBECFEFD4E02A
:10007000DEBFCDBF11E0A0E0B1E0E8EEF3E002C0EA
:1000800005900D92A230B107D9F711E0A2E0B1E0DE
:1000900001C01D92A431B107E1F70E94AF010C9499
:1000A000F3010C94000082958F708A302CF4805DEF
:1000B000992787FD90950895895C992787FD9095EC
:1000C00008958F708A302CF4805D992787FD909574
:1000D0000895895C992787FD909508958A332CF4BB
:1000E0008053992787FD909508958753992787FD19
:1000F00090950895EF92FF921F93162F0E946E0025
:10010000E82EFF24E7FCF094E294F29480EFF822CA
:10011000FE24E822FE24812F0E946E008E2999275A
:1001200087FD90951F91FF90EF90089588E180934F
:10013000C10086E08093C20089E18093C4001092E0
:10014000C5000895982F8091C00085FFFCCF909343
:10015000C60008958091C00087FFFCCF8091C60043
:10016000992787FD909508951092640080E480930C
:100170007C008BEC80937A00109213011092120194
:100180008DED809302018EEE80930A0121E030E034
:10019000F901EE5FFE4F8DED8083F901E65FFE4FC2
:1001A0008EEE80832F5F3F4F2830310589F7089509
:1001B0001F920F920FB60F9211242F933F938F939C
:1001C000EF93FF93209112013091130180917800F9
:1001D000F901E65FFE4F808380917900F901EE5FBF
:1001E000FE4F8083273031053CF42F5F3F4F309323
:1001F00013012093120104C01092130110921201F6
:1002000080911201806480937C0080917A008064E8
:1002100080937A00FF91EF918F913F912F910F90F2
:100220000FBE0F901F901895FC0185E580836295A5
:10023000607F4F70462B4183832F992787FD9A95C6
:10024000828323830895FC0185E580836295607F26
:100250004F70462B4183832F992787FD9A95828380
:10026000238308950F93FC0185E580836295607F69
:100270004F70462B418322830383022704830F910F
:1002800008950F93FC0185E580836295607F4F7030
:10029000462B418322830383022704830F91089511
:1002A000FC012FEF3FEF348723878CED95E0928799
:1002B0008187308727830895FC012FEF3FEF348734
:1002C00023878CED95E09287818730872783089577
:1002D0000F931F93CF93DF93EC010E94AA00853503
:1002E000E1F70E94AA00282F22952F7033273C8720
:1002F0002B87992787FD90958F70907098878F83B3
:100300000E94AA00082F0E94AA00182F0E94AA008B
:10031000E82F8B859C85892BE9F4F894602F77274B
:1003200067FD7095412F552747FD50959A01262767
:1003300037278E2F992787FD90952817390711F0B9
:10034000789408C0962F88275070842B952B9A8715
:100350008987F6CFDF91CF911F910F910895C2EF5A
:10036000D4E0DEBFCDBF0E94B4000E949600789416
:10037000EE24FF245E010894A11CB11C26E0C22ECD
:10038000D12CCC0EDD1EF701EE5FFE4F0081112750
:1003900007FD1095102F0027F701E65FFE4F8081C3
:1003A0009927082B192B8091000190910101080FCA
:1003B000191F212F3327A70160E0C5010E944101C9
:1003C0008501F80181918F010E94A2000C151D0585
:1003D000C1F70894E11CF11CF8E0EF16F1049CF25F
:0803E000EE24FF24D0CFFFCF73
:0203E800E80328
:00000001FF
